:020000040000FA
:10000000000005308A00092DFF0003088301FE006F
:100010000A088A01FD000408FC0083017C088400B2
:100020007D088A007E088300FF0E7F0E0900A00174
:10003000A101A201A301612817208528172071289A
:100040001E201E201E28073083169F0083124F306B
:10005000F0000530F1002C30F4004830F3000800C7
:100060003A208A01F50005308A001230750703181E
:100070008A0A8200F00A0319F10A71088A007008DE
:1000800082003A208A01FB003A208A01FA006128A6
:100090007A1C53288B1C53288B10A5200930F100A3
:1000A0005230F00054286128302054286400630046
:1000B0005628FC30F4076128F403F40361282C303F
:1000C000F40083136400080008002C30F40083134C
:1000D00008306D208A110A12102DFF3E031D6D207D
:1000E00008007408840020088000840A2108800029
:1000F000F40AF40A6128F403F40374088400000885
:10010000A000840A0008A100612874088400200867
:100110008000840A21088000840A22088000840A62
:10012000230880000430F4076128FC30F4077408C9
:1001300084000008A000840A0008A100840A0008C6
:10014000A200840A0008A3006128F303F3037308E4
:10015000840070088000840A710880006128730898
:1001600084000008F000840A0008F100F30AF30A92
:10017000612800080800CB20B928CD20B928CF205D
:10018000B928D120B92884000308F700740884072F
:10019000770883000800FF30C328FE30C328FD30F5
:1001A000C328FC30C3283A208A01F5003A208A018E
:1001B000F0007508F1005F28A5203A208A01F500BB
:1001C0003A208A01F0007508F1006128AF20672805
:1001D000AF200230F0070318F10A61282008031D40
:1001E000D328E92820080319D328E928FE3EF50082
:1001F00000300318013E8A00750882000134023481
:1002000004340834103420344034803401308A00FF
:100210000D302D0703188A0A82000534063407348E
:100220000534053405340534053438302C05AD006B
:100230000310AD0DAD0E062184002C080739F628F9
:1002400015218417FF3A8005FF3A841380040800C3
:1002500020215F2815218417FF3A8005841380052B
:1002600008002A215F2815218417800484130800C0
:1002700033215F2815218417FF3A8005FF3A841344
:1002800008003A215F28A301A2013A208A01A100B7
:100290003A208A01A0006128A301A201A1013A200D
:1002A0008A01A00061284C2171284C218528432116
:1002B0007128432185287508A0070318A10A76082C
:1002C000A10708000130A10576187E29F51B7229C7
:1002D00021186E2920086F3C031808003030A00751
:1002E00003182114211878292008EF3C031808006E
:1002F00021142030A007031821148029F51B0800C1
:1003000020086F3C031808002030A00703182114B0
:1003100008005B2162210830A10461280310A00DB0
:10032000A10D5B2162210630A10461280310A10CFC
:10033000A00C10300318F6075B210311F61AA00A6F
:100340000319A10A6221103076050438A10461283E
:100350000310A10CA00C10300318F6070310A10C19
:10036000A00C20300318F6070310A10CA00C40309D
:100370000318F6075B210311F61BA00A0319A10A53
:100380006221703076050238A104612876080E39A2
:10039000023C0319A82976080E39043C0319962952
:1003A00076080E39083C0319892976080E39063C6F
:1003B00003198E296128211883172008840000085A
:1003C000A000A101A201A301612821188317200820
:1003D00084000008A000840A0008A100A201A30173
:1003E00061282108F50075188317200884000F3054
:1003F000751AF0300005A000A101A201A301751A31
:10040000A00E61282108F5007518831720088400C4
:10041000210E0739F620A0010005031D2014A101BB
:10042000A201A301612821188317200884002C0849
:100430008000612821188317200884002C08800080
:10044000840A2D0880006128211883172008840061
:100450000F30AC05211EF03080052C08211A2C0E1F
:10046000800461282118831720088400210E073991
:10047000F6208004FF3A2C1C8005612821080E39E3
:10048000023C0319022A21080E39043C0319F12900
:1004900021080E39083C0319DB2921080E39063CD6
:1004A0000319E5293A208A01A100F6003A208A01C1
:1004B000A000F61F5F2AF613F5009520C6296128D3
:1004C0005222712852223E2A6222712862228528F5
:1004D00021080E39023C0319322A21080E39043C46
:1004E0000319242A21080E39083C0319132A21086C
:1004F0000E39063C03191A2A612868225F28A009D0
:10050000A109A209A309A00A0319A10A0319A20AB1
:100510000319A30A61282030F500A401A501A60152
:10052000A701A801283084000530F60064003330AC
:1005300080078019F039801B0F3980028403F60B85
:10054000962AA00DA10DA20DA30DA40DA50DA60D1B
:10055000A70DA80DF50B922A6128C120A004BF2089
:10056000A104BD20A204BB20A3045928C120A007D8
:10057000BF200318013E031DA107BD200318013E43
:10058000031DA207BB200318013E031DA30708009B
:10059000B62259287F22C82AC120A400BF20A50066
:1005A000BD20A600BB20A700A801A901AA01AB019C
:1005B0002130F500A30CA20CA10CA00CF50303192B
:1005C0006128031CF12A2408A80725080318013E06
:1005D000A90726080318013EAA0727080318013EA9
:1005E000AB07AB0CAA0CA90CA80CDA2ACC22592810
:1005F000FF30A000A100A200A3000800A001A101FB
:10060000A201A3010800031DF8220319FE225928A4
:10061000BB20F500230203191A2B75082306803925
:100620000319162B0310A31B282B2A2B7508230252
:10063000031D282BBD202202031D282BBF202102D1
:10064000031D282BC1202002031D282B0230080087
:10065000013003180430080008230439032B082351
:100660000639032B08230239032B08230139032BF6
:100670002908A000A1012408F5002508F600C621DC
:100680003E2AA80EF030A805A70E0F302705A804B3
:10069000F030A705A60E0F302605A704F030A605FA
:1006A000A50E0F302505A604F030A505A40E0F30C9
:1006B0002405A504F030A4050800A000A101A201B2
:1006C000A3012B083228A800281C6D2B3A208A0190
:1006D000A000A101A201A301842BA81C782B3A2021
:1006E0008A01A1003A208A01A000A201A301842B63
:1006F0003A208A01A3003A208A01A2003A208A0106
:10070000A1003A208A01A0002B083220A90BAA0AD6
:10071000AA0B642B61283A208A01AB003A208A0197
:10072000013EAA003A208A01A90008007B20200887
:10073000A8007B202008A600210AA7007B20200813
:10074000A4002108A5003A208A01AB00A9010800F5
:100750003A208A01AA003A208A01AB0008009520BD
:10076000AA1F0800A31F08007F2285202D305D23CB
:10077000952008003F30AA050A30A9002A0829025E
:100780000319C52B4123A90BBE2B77082A02031995
:10079000D22B280E0F39031DD42B4123AA0BC52BB6
:1007A000AA0AA801280E0F39A900F63E3030031816
:1007B000373029075D234123AA0BD22B61288520DE
:1007C000A823AF238B22BA2B2008F7009520DF2B1C
:1007D0008B230130632B8B230230632B962338232A
:1007E0002B083220A90AA60BA70AA70BEF2B61281A
:1007F000AD0A1E3EAC020318AD0AAD0B252CAC09A8
:1008000004308A002C0A063E03188A0A820000007F
:1008100000000000000000000000000000000000D8
:100820000800080008000800080008000800080088
:100830000800080008000800080008000800080078
:100840000800080008000800080064000A30AC0234
:100850000318AD0AAD030319FF2B252C0301F82360
:100860005F28A10A6400DD30AC000330AD000C301D
:10087000F823A00BA10AA10B322C080031245F2819
:100880001521841780048413AF0000052E1C2F0649
:100890000319612C34088400300803196B2C0008FC
:1008A000031D592C0130A000A1013E243008800016
:1008B0006B2C800B662C300A03196B2C32088000DD
:1008C0006B2C340884003518831780010230F00740
:1008D0000318F10A5F28D32883132C308400443096
:1008E000A0008524A03084005030A0008524103062
:1008F000840083176030A000852490308400831723
:100900006030A00085248313612864008001840A7C
:10091000A00B852C0800300803178D008F0183166B
:100920008C130C140000000083120C080313AC009D
:10093000AD01AE01AF01B00A08008B2468225F2828
:10094000300803178D008F010313200803178C0054
:1009500083168C130C1555308D00AA308D008C1425
:1009600064008C18B02C0C1183120313B00A080019
:10097000A0245F28A0246128B100340A0319C32CE5
:100980003408AC002A213008AC00B11B2A21B11F69
:10099000332136088400F030371A0F308417800571
:1009A000841380053108371A310E371E0F39371A74
:1009B000F03980043208AC0020212830AC00AD01B1
:1009C0000301F8233208AC002A210800200E0F3959
:1009D00021188038BC2420080F3921188038BC2405
:1009E000211C612804302002031861288830AC00E3
:1009F0001330AD000301F82361288316010583122B
:100A00002C04810164008316810083125F28BF30AB
:100A1000FD2C2320831603138E180F2D8E148312A2
:100A20003020102D642871287B2885289528562889
:100A30005628A528AF28602A522A662A642A622AE4
:100A4000552953294C295929572943297D2A5F289B
:100A5000202821281E281C2817286C2CAD2AF62AAD
:100A6000C82ACA2A7F2A2C2B2F2B322B352BEE2873
:100A7000F228D328DC28E628E828402C2829312928
:100A8000382941293E2C2E2C9D2C8B2CB82CBA2C8D
:100A9000E42BE82BEB2BEE2BE62C072D48284128E6
:100AA00018342E340F3401342F340F3402342F34E1
:100AB0000F3403342F340F3404342F340F340534FF
:100AC0002F340F3408342E340F3409342F340F34BC
:100AD0000A342E340F340B342F340F340C342E34AC
:100AE0000F340D342E340F340E342F340F340F34B2
:100AF0002F340F3410342F340F3411342F340F347B
:100B000012342F340F3413342F340F3414342F3461
:100B10000F3415342F340F3416342F340F34173468
:100B20002F343D34003401343C340F3440343B34F2
:100B30003C3412340134F43430343C3417340F3440
:100B400005340F3403340F340434093414340734B7
:100B500038343A3400340634013403340134023476
:100B600001342834013401340134023401340C34AA
:100B700015343C3417340F3405340F3403340F3438
:100B8000043409341434073438343A34003411341A
:100B900001340134013402340034533400346834F5
:100BA00000346F340034743400344D340034653410
:100BB000003474340034653400347234003420342A
:100BC0000034493400345634003420340034623464
:100BD00000347934113401348034103440341E34FC
:100BE0003A3437343A3400340E345234693463348E
:100BF000683420344B346134703470346D3465346F
:100C000069346534723415343C340F3413342C3465
:100C10003C3412340134F43430343C340F34133463
:100C20002D343C340F3409342C343C341234013428
:100C3000F43430343C340F3409342D343C341B3418
:100C40003C340E3420340A3408345F3414343C34D9
:100C50000E3420340A340834603414343C341634EE
:100C6000093408345A3432343C3417340F340134E4
:100C7000093408345B3432343C3417340F340234D2
:100C8000093408345C3432343C3417340F340334C0
:100C900009340834513432343C3417340F340434BA
:100CA00009340834503432343C3417340F340534AA
:100CB000093408345D3432343C3417340F3406348C
:100CC000093408345E3432343C3417340F3407347A
:100CD00009340834553432343C3417340F34083472
:100CE00009340834543432343C3417340F34093462
:100CF00009340834533432343C3417340F340A3452
:100D000009340834523432343C3428340E34F33449
:100D10003C3417340F3405340F3403340F340434A7
:100D200009341434073438343A340034123401347A
:100D300001340134023400342034003443340034AC
:100D40006C3400346534003461340034723400345F
:100D50002034003456340034613400346C340034B0
:100D60007534003465340034733400342D34003469
:100D70002D3400343E341134013480341034403486
:100D80001E343A3437343A340034103420342034AA
:100D900020345334653474347534703420342F3433
:100DA00020345334743461347234743415343C3424
:100DB0000F340C340F3401340F34FF340F34023449
:100DC00009341234A1340F3401342B3407345B342A
:100DD0003C340F340A340F3401340F34FF340F34F1
:100DE000023409342234A1340F3401342B34093451
:100DF0006D343C340F340D340F3401340F34FF3470
:100E00000F34023409343234A1340F3401342B341A
:100E1000073411343C340F34C83430343C34273474
:100E20000634D6343C340B3408345A340A3408348B
:100E30005E3414343C3419340A34063454341434D3
:100E40003C3419340A340634523414343C341734E4
:100E50000F3405340F3403340F340434093414349C
:100E6000073438343A340034113401340134013455
:100E70000234003456340034613400346C340034AD
:100E80007534003465340034733400342034003455
:100E9000433400346C34003465340034613400343D
:100EA0007234003465340034643400342134153431
:100EB0003C342734063483343C3428340E34F33441
:100EC0003C3417340F3405340F3403340F340434F6
:100ED0000934143407341334013402343A340D34F1
:100EE00008345F343A3437343A340034053420342B
:100EF00020342034203420340B3408345E34103451
:100F0000033436340A343A3437343A34003406344D
:100F10002034203420342034203420340D3408345C
:100F200060343A34113401348034103440341E3487
:100F30003A3437343A340034023454343A340B34CB
:100F4000063454341034043436340A343A343734E2
:100F50003A34003406342034203420342034F6343B
:100F60003A340B34063452341034043436340A34F0
:100F70003A3415343C340F340C340F3401340F340C
:100F8000FF340F34023409341234A1340F340134E5
:100F90002B340834ED343C340F340A340F3401342C
:100FA0000F34FF340F34023409342234A1340F34A7
:100FB00001342B34093423343C340F340D340F34D2
:100FC00001340F34FF340F34023409343234A13485
:100FD0000F3401342B3409343A343C340B340634A6
:100FE00048341A34233426340734FC343C340F3468
:100FF00009342D342734083408343C340B34063497
:101000004834103401341F3403340A34063448346D
:1010100014343C340B3406344A341A342334263422
:10102000083418343C340F3413342D342734083446
:1010300024343C340B3406344A34103401341F3425
:1010400003340A3406344A3414343C340B34023446
:1010500005341A34233425340D34FB343C340B343A
:10106000083458341A34233425340734B9343C3422
:101070000B34083459340D34083458341E340334D6
:101080000A340834593414343C3419340A340834DA
:10109000583414343C340B3422345D340A34123462
:1010A000063414343C340B34063452340D340834D2
:1010B00059341E3403340A340634523414343C3464
:1010C0000B34063454340D34083459341E3403348C
:1010D0000A340634543414343C340B3408345E344B
:1010E0001A3424342634083481343C340B34083424
:1010F0005E340D34083459341F3403340A34083450
:101100005E3414343C3419340A34083459341434F9
:101110003C340B3408345E340D3408345A342434EF
:101120002634083498343C3419340A3408345E3494
:1011300014343C340B3408345E340D3408345B34DE
:10114000213426340834BE343C340E344C340A3452
:1011500008345F3414343C340B34063448341034CF
:10116000C8341E3403340A3406344A3414343C344C
:101170000B3402345D340A343234073414343C34D2
:101180000B34063454340D340634503424342634AD
:101190000834E9343C340E3454340A3408346034AE
:1011A00014343C340B34063448341034C8341E3400
:1011B00003340A3406344A3414343C340B341234C5
:1011C0005D340D3402345D341C3403340A3432345B
:1011D000073414343C34273407345F343C34283427
:1011E0000E34F3343C340B3408345E340B3408349E
:1011F0005A340D3408345C341F3424342634093412
:101200000B343C340B3408345A340A3408345E341A
:1012100014342734093418343C340B3408345C3427
:101220000D3408345E341E3403340A3408345E341A
:1012300014343C340E3420340A3408345F3414340B
:101240003C34273407345F343C3428340E34F334D0
:101250003C340B3408345A340A3408345E341434C1
:101260003C340E3420340A3408345F3414343C34B3
:10127000273407345F343C3428340E34F3343C34A0
:1012800019340A340634543414343C340E342034C3
:101290000A340834603414343C34273407345F345F
:1012A0003D34003400340B340834583410340134E5
:1012B0001E3403340A340834583414340B341434D0
:1012C0005D34103401341E340334103419341D34A9
:1012D00003340A34063448341434293428340E34A0
:1012E000F3340B3408345A341034AA3424342634FA
:1012F00009347F340E34AA340A3408345A3414348E
:101300000B3408345A340A3406344C3414340E3452
:10131000FA340A3406344E3414340E3405340A34A4
:1013200008345734143417340F3405340F3403346D
:101330000F34043409341434073438343A34003464
:101340001134013401340134023400344C3400349B
:101350006F34003461340034643400346534003454
:1013600072340034203400344334003461340034A7
:101370007034003461340034633400346934003430
:10138000743400347934153428340E344D34283410
:101390000E3468340B340234A1341A342334253427
:1013A0000934C3340B3406344C340A3408345A3408
:1013B00014340B3408345B340D3408345A34243478
:1013C00026340934E9340B3408345A340A340834E6
:1013D0005B3414340B3408345B340A3406344C3434
:1013E00014340B3408345A340A3406344E3414346A
:1013F0000E3405340A3408345734143417340F3497
:1014000005340F3403340F340434093414340734EE
:1014100038343A34003410340134013401340234A5
:1014200000344C3400346F3400346134003464349C
:1014300000346534003472340034203400345434C1
:101440000034723400346934003467340034673453
:101450000034653400347234153428340E344D347D
:1014600028340E3468340B340234A1341A34233453
:1014700025340A342C340B3406344C340A34083402
:101480005B3414340B3408345C3410346434243446
:1014900026340A3450340E3464340A3408345C344C
:1014A00014340B3408345C340A3406344C341434A9
:1014B0000E34C8340A3406344E3414340E34053431
:1014C0000A3408345734143417340F3405340F34C5
:1014D00003340F34043409341434073438343A34C0
:1014E00000340E34013401340134023400345034F9
:1014F00000346F3400346434003420340034433416
:1015000000346134003470340034613400346334A6
:101510000034693400347434003479341534283498
:101520000E344D3428340E3468340B340234A13474
:101530001A34233425340A348E340B3406344C34B4
:101540000A3408345C3414340B34063450340A340E
:1015500006344C34143411340734D0340A3406348D
:101560004E3414340E3432340A34083457341434BC
:101570000B3406344C3413340734D034243426343A
:101580000A34C8341134013490340A3406344C34EB
:10159000143417340F3405340F3403340F34043447
:1015A00009341434073438343A3400340E340134F6
:1015B00001340134023400345434003461340034D2
:1015C0006E3400346B34003420340034543400342E
:1015D00072340034693400346734003467340034C2
:1015E000653400347234153417340F3405340F3435
:1015F00003340F34043409341434073411340134FF
:101600008034103440341E343A340B3406344C34B5
:101610001034043436340A343A34153428340E3451
:1016200068340B340234A1341A34233425340A3498
:10163000F3340B3406344C340A3406345034143446
:101640000B3402345D3410340134233426340B342B
:1016500031340E3459340A3406344C3414342734BB
:101660000B3437340E344E340A3406344C341434CC
:1016700028340E34F33417340F3405340F34033464
:101680000F34043409341434073438343A34003411
:101690001034013401340134023400344C34003449
:1016A0006F34003461340034643400346534003401
:1016B0007234003420340034413400347534003442
:1016C00064340034693400346F3400343A34003404
:1016D00020340D3406344C343A3415340F340C3481
:1016E0000F3401340F34FE340F3402340934123411
:1016F000A1340F3401342B340B34AE340F340A349C
:101700000F3401340F34FE340F34023409342234E0
:10171000A1340F3401342B340B34A0340F340D3486
:101720000F3401340F34FE340F34023409343234B0
:10173000A1340F3401342B340B34BD3427340B3433
:101740006D340E344E340A3406344C3414341934A7
:101750000A3402345D34143427340B3437340E34F5
:1017600059340A3406344C3414340E3401340A34F7
:1017700002345D34143427340B3437340B341234D0
:101780005D3410340134233426340B34CF340E341A
:1017900059340A3406344C34143427340B34D534D9
:1017A0000E344E340A3406344C34143428340E3497
:1017B000F33417340F3405340F3403340F34043446
:1017C00009341434073438343A3400340E340134D4
:1017D00001340134023400345434003461340034B0
:1017E0006E3400346B34003420340034413400341F
:1017F0007534003464340034693400346F34003498
:101800003A34003420340D3406344C343A34153430
:101810000F340C340F3401340F34FE340F340234DF
:1018200009341234A1340F3401342B340C344834CD
:101830000F340A340F3401340F34FE340F340234C1
:1018400009342234A1340F3401342B340C343A34AB
:101850000F340D340F3401340F34FE340F3402349E
:1018600009343234A1340F3401342B340C3457345E
:1018700027340C3407340E344E340A3406344C34D6
:10188000143419340A3412345D34143427340B34CC
:10189000D5340E3459340A3406344C3414340E34EE
:1018A00001340A3412345D34143427340B34D53403
:1018B0000B3422345D3410340134233426340C3498
:1018C00069340E3459340A3406344C341434273411
:1018D0000C346F340E344E340A3406344C34143421
:1018E00028340E34F33417340F3405340F340334F2
:1018F0000F34043409341434073438343A3400349F
:101900000D340134013401340234003441340034E4
:101910006734003469340034743400346134003482
:1019200074340034693400346F3400346E3400345D
:101930003A34003420340D3406344C343A341534FF
:101940000F340C340F3401340F34FE340F340234AE
:1019500009341234A1340F3401342B340C34E03404
:101960000F340A340F3401340F34FE340F34023490
:1019700009342234A1340F3401342B340C34D234E2
:101980000F340D340F3401340F34FE340F3402346D
:1019900009343234A1340F3401342B340C34EF3495
:1019A00027340C349F340E344E340A3406344C340D
:1019B000143419340A3422345D34143427340C348A
:1019C0006F340E3459340A3406344C3414340E3423
:1019D00001340A3422345D34143427340C346F3427
:1019E00028340E34F33417340F3405340F340334F1
:1019F0000F34043409341434073438343A3400349E
:101A00000F340134013401340234003450340034D2
:101A1000753400346C34003473340034653400346D
:101A2000203400344C340034653400346E340034D7
:101A30006734003474340034683400343A34153474
:101A40000B3414345D340A3406344C3414340E34FC
:101A50000F340A3406344E3414340E3401340A344C
:101A600008345734143419340A34083456341434CE
:101A70000B34083456340D3406344C3422342634B6
:101A80000D344D340E34FF340B34083456340A34DC
:101A900088346134143427340D3456340E342D34E4
:101AA0000B34083456340A348834613414340B341B
:101AB00008345634103401341E3403340A340834E4
:101AC000563414340B340834563410341034213462
:101AD00025340D34373419340A3408345634143468
:101AE00017340F3405340F3403340F3404340934FD
:101AF00014340734113401348034103440341E342B
:101B00003A340934083461340F3410341834393419
:101B10003A34153428340E3468340B340234A1348A
:101B20001A34233425340D3437340B3406344C3412
:101B30000A3414345D34143416340C3408345A34F2
:101B4000343417340F3401340C3408345B343434F7
:101B500017340F3402340C3408345C343434173402
:101B60000F3403340C3408345134343417340F3404
:101B700004340C3408345034343417340F340534FE
:101B80000C3408345D34343417340F3405340F34D6
:101B900003340F34043409341434073438343A34F9
:101BA000003411340134013401340234003453342C
:101BB00000346134003476340034693400346E34D7
:101BC00000346734003420340034653400346E341B
:101BD00000347434003472340034693400346534B1
:101BE0000034733400342134153412340134F434A5
:101BF0003034273406341F3417340F3406340D3490
:101C000008345E3435340D340834553435340D34ED
:101C10000834543435340D340834533435340D34E9
:101C2000083452343534153417340F3405340F3436
:101C300003340F34043409341434073438343A3458
:101C400000341234013401340134023400342034BD
:101C50000034423400346134003474340034743459
:101C60000034653400347234003479340034203464
:101C7000003420340034443400346534003461349A
:101C800000346434003421340034203415340F34EB
:101C900009342D340F3413342D34063417340F34F3
:101CA00005340F3403340F34043409341434073446
:101CB000113401348034103440341E343A340B343F
:101CC00006344C341034033436340A343A34153480
:101CD0002A340F340C340F3401340F34FF340F34F2
:101CE000023409341234A1340F3401342B340E344D
:101CF0009B340F340A340F3401340F34FF340F3463
:101D0000023409342234A1340F3401342B340E341C
:101D1000C1340F340D340F3401340F34FF340F3419
:101D2000023409343234A1340F3401342B340E34EC
:101D3000E93427340E34683428340E34F3340B3449
:101D400006344C340D34083457341E3403340A340A
:101D500006344C3414340B3406344C340D3406340D
:101D60004E34243426340E34B93419340A3406344B
:101D70004C34143419340A340234A1341434273462
:101D80000E34F23428340E34F3340B3406344C342D
:101D90000D34083457341F3403340A3406344C34B9
:101DA00014340B3406344C340D3406344E3424349D
:101DB00026340E34E1340B3406344E340A340634FF
:101DC0004C34143419340A340234A1341434273412
:101DD0000E34F23428340E34F3340E3401340A3421
:101DE0000234A13414342A340F3413342C340B3419
:101DF0004234063410340134233426340F34023490
:101E000027340E34F6340B342234063410340134C3
:101E1000233426340F340E3427340F3402340B3479
:101E20005234063410340134233426340F341A3437
:101E300027340F340E340F34323430340F3413342B
:0C1E40002D340F34643430342A3406345E
:02400E00753FFC
:00000001FF
